:100000000C9483000C94B5260C94E0260C940B27DA
:100010000C94AF000C94AF000C94AF000C94AF00A4
:100020000C94AF000C94AF000C94AF000C94AF0094
:100030000C94AF000C94AF000C94AF000C94AF0084
:100040000C94AF000C94AF000C945C280C94AF009F
:100050000C94C32B0C94F92B0C94AF000C94AF00B0
:100060000C94AF000C94AF000C94AF000C94AF0054
:100070000C94AF000C94AF000C94AF000C94F924D6
:100080000C94AF000C94AF000C94AF000000000182
:100090000200090A00000000040308070000000035
:1000A0000000000000000000000000000102040841
:1000B0001020408001020408102040800102040842
:1000C0001020408001020408102040800202020239
:1000D00002020202040404040404040403030303EC
:1000E00003030303010101010101010100002200DA
:1000F000250028002B0000002100240027002A00F2
:10010000CA05811D2D2C2092DC3911241FBECFEF92
:10011000D0E4DEBFCDBF11E0A0E0B1E0EAE6F0E65A
:1001200000E00BBF02C007900D92AA3AB107D9F7C1
:1001300029E3AAEAB1E001C01D92AC3DB207E1F7A4
:1001400010E0C3E8D0E004C02197FE010E946E2EAB
:10015000C038D107C9F70E94B02C0C9433300C94EE
:100160000000CF93DF931F92CDB7DEB76983DC0128
:10017000ED91FC910280F381E02D41E050E0BE0161
:100180006F5F7F4F09950F90DF91CF91089508958C
:10019000FC011382128288EE93E0A0E0B0E0848339
:1001A0009583A683B78389E491E09183808380E57A
:1001B000848781E085878AE090E09787868789E059
:1001C00090E0918B808B82E090E0938B828B148AFD
:1001D000158A168A178A118E108E138E128E158E1E
:1001E000148E40E050E0BA01CF010C94872CFC0142
:1001F00077876687518B408B338B228B08950F93C3
:100200001F93CF93DF93EC01062F142F60E08E85B0
:100210000E94622A3C852D8580913039882381F0A7
:100220009FB7F89480913039813081F58DB38093F8
:100230002E394DB380912F39809584238DBB9FBF7C
:100240003CBD2DBD0EBD00000DB407FEFDCF8EB52B
:100250001EBD00000DB407FEFDCF1EB580913039E4
:10026000882351F09FB7F8942091303980912E392E
:10027000213079F48DBB9FBF61E08E850E94622A98
:10028000812FDF91CF911F910F91089590932E3977
:10029000D7CF8FBFF1CF6F7740E00C94FF0068E1BC
:1002A0000C944B0169E10C944B0169E10E944B01F4
:1002B000682F880F770B880B990B0E94FC2C20E08D
:1002C00030E040E85EE30E94AC2D08958F929F924B
:1002D000AF92BF92EF92FF920F931F93CF93DF9352
:1002E0008C016AE10E944B01C82FD0E0C8010E9436
:1002F00055010E94C42C4B017B01F801648975896A
:10030000868997890E94FC2C24ED30E843E45EE462
:100310000E94BF2CBE0187FD12C06D597109F7FE06
:1003200011C0680D791DCB01DF91CF911F910F9105
:10033000FF90EF90BF90AF909F908F900895645A78
:100340007109EDCF072E000C880B990B0E94FC2C35
:1003500020EB32E748E85FE30E94AC2D0E94C42CFA
:10036000E2CFCF93DF93EC0163E10E944B0190E079
:10037000288D398D821B930BDF91CF910895CF93F8
:10038000DF93EC01E881F9810480F581E02D099586
:10039000892B69F0888D998D0196998F888F60E0FF
:1003A000CE010E944B0190E0DF91CF9108958FEF35
:1003B0009FEFFACF0F931F93CF93DF938C0166E0EB
:1003C0000E944B01D82F67E0C8010E944B01C82F43
:1003D00068E0C8010E944B014C2F50E070E060E0E3
:1003E000762F652F542F44276D2B8A019B01082BF4
:1003F000C901B80120E038E448EE51E00E94892E9E
:1004000003E10E942E2FB901CA01DF91CF911F9104
:100410000F9108956DE10E944B0190E034E09595B5
:1004200087953A95E1F78A30910574F4FC01EE0F57
:10043000FF1FE80FF91FE95DFE4F60817181828126
:10044000082E000C990B089560E070E0CB01089530
:100450006CE20C944B01CF93DF93EC0143E861E82D
:100460000E94FF0062E1CE010E944B0183FD03C0A8
:100470000E945B28F7CF48E062E9CE010E94FF00AE
:1004800081E090E0DF91CF910895AF92BF92CF923B
:10049000DF92FF920F931F93CF93DF936C015B0169
:1004A000EA0162E20E944B01F82E90E09C012C0FC1
:1004B0003D1F2F3F310529F020F0CFEFD0E0C81BC2
:1004C000D90B8501AC0EBD1E0A151B0541F0F801C4
:1004D00041918F0160E8C6010E94FF00F5CF4C2FCB
:1004E0004F0D62EAC6010E94FF00CE01DF91CF915D
:1004F0001F910F91FF90DF90CF90BF90AF90089524
:100500000F931F93CF93DF93EC01E881F98104806F
:10051000F581E02D0995892BB1F06DE0CE010E94A7
:100520004B01082F60E0CE010E944B01182F402F95
:100530006DE8CE010E94FF00812F90E0DF91CF9106
:100540001F910F9108958FEF9FEFF8CFCF93DF9317
:10055000EC017D8F6C8F8A899B89672BA1F160E00C
:100560000E94262A40E060ECCE010E94FF008A89AA
:100570009B8982309105D9F08A309105D1F00B9793
:10058000D1F481E00E9435268A899B8982309105C9
:10059000A1F08A30910599F00B9799F481E043E03E
:1005A00050E06AEA75E0DF91CF910C94702682E00A
:1005B000E9CF80E0E7CF8FEFE5CF82E0F0CF80E0BA
:1005C000EECF8FEFECCF82309105B9F08A309105F4
:1005D000B1F00B97B1F481E00E949F268A899B8934
:1005E0008230910581F08A30910579F00B9779F48A
:1005F00081E0DF91CF910C94542682E0EDCF80E032
:10060000EBCF8FEFE9CF82E0F4CF80E0F2CF8FEF36
:10061000F0CF41E861E80C94FF0040E861E80C94F9
:10062000FF000E940D030C942126AF92BF92CF923F
:10063000DF92EF92FF920F931F93CF93DF93EC0122
:10064000DB01CA018C8B9D8BAE8BBF8B6A017B015A
:10065000FF0CCC08DC2C76019A01AB016C2D7C2DB3
:100660008C2D9C2D03E10E94132FA12CE8E4BE2EBB
:10067000F8EECF2EDD24D394E12CF12C00E010E035
:100680000E94B62E122FC22ED32E7A01A701662702
:10069000772766E8CE010E94FF0077276F2D5E2D39
:1006A0004D2D67E8CE010E94FF00412F68E8CE0182
:1006B000DF91CF911F910F91FF90EF90DF90CF903E
:1006C000BF90AF900C94FF00CF92DF92EF92FF9219
:1006D000CF93DF93EC016A017B0161E08E850E947C
:1006E000262A61E08E850E94622A888999898F3F37
:1006F0009807B9F061E00E94262A60E088890E948C
:10070000622A6AE070E080E090E00E94D72861E011
:1007100088890E94622A6AE070E080E090E00E948E
:10072000D7280E94EB2562E4CE010E944B01823162
:1007300091F5CE010E940D03B701A601CE010E94E2
:10074000150340E06EE8CE010E94FF0040E06FE834
:10075000CE010E94FF006CE0CE010E944B01482FA9
:1007600043606CE8CE010E94FF0044E066EACE01DF
:100770000E94FF0040E869E8CE010E94FF00CE0120
:100780000E94090381E090E0DF91CF91FF90EF900C
:10079000DF90CF90089590E080E0F6CFCF92DF9287
:1007A000EF92FF92CF93DF93EC016EE10E944B0139
:1007B000F82ECE010E940A02F2942FE0F222CC24FD
:1007C000C394D12C02C0CC0CDD1CFA94E2F70D2CA2
:1007D000000CEE08FF0828EE33E040E050E00E94F5
:1007E0004F2EC701B6010E944F2E21313105410520
:1007F00051055CF04CE066EACE01DF91CF91FF90AD
:10080000EF90DF90CF900C94FF0044E0F4CF0F9373
:100810001F93CF93DF938C01EB016630710534F0A9
:100820006D30710534F56630710529F545EC61EBE5
:10083000C8010E94FF004CE067EBC8010E94FF0066
:10084000C6E0D0E06EE1C8010E944B018F7094E0D9
:10085000CC0FDD1F9A95E1F74C2F482B6EE9C801AC
:100860000E94FF00C801DF91CF911F910F910C945E
:10087000CE03CCE0D0E043EC61EBC8010E94FF0066
:100880004AE067EBC8010E94FF00DCCFCF92DF9205
:10089000EF92FF920F931F93CF93DF938C01CB01C5
:1008A000BA010E94FC2C6B017C0120E030EC43EF8C
:1008B00055E40E94BF2CD0E0C0E018160CF065C0D3
:1008C00020E030E842E256E4C701B6010E94BF2CA6
:1008D000C1E0D0E018160CF058C020E030EC43E73F
:1008E00056E4C701B6010E94BF2CC2E0D0E0181642
:1008F0000CF04BC020E030E842EA56E4C701B601F4
:100900000E94BF2CC3E0D0E018160CF03EC020E0DF
:1009100034E244EF56E4C701B6010E94BF2CC4E0A4
:10092000D0E0181694F520E034EE42E257E4C70117
:10093000B6010E94BF2CC5E0D0E0181634F520E0C7
:1009400034E244E757E4C701B6010E94BF2CC6E079
:10095000D0E01816D4F420E034E244EF57E4C701A5
:10096000B6010E94BF2CC7E0D0E0181674F420E056
:1009700034E244E758E4C701B6010E94BF2CC9E045
:10098000D0E0181614F0C8E0D0E06DE1C8010E9474
:100990004B018F7094E0CC0FDD1F9A95E1F74C2F3F
:1009A000482B6DE9C8010E94FF00C801DF91CF917B
:1009B0001F910F91FF90EF90DF90CF900C94CE039A
:1009C0000F931F93CF93DF938C01EB016930710577
:1009D00014F0C8E0D0E06DE1C8010E944B01C530C1
:1009E000D10514F4C5E0D0E02497CC0FDD1F482FCB
:1009F000417F4C2B6DE9C801DF91CF911F910F9181
:100A00000C94FF00CF93DF93EC016EE10E944B0149
:100A1000482F44606EE9CE01DF91CF910C94FF0026
:100A2000CF93DF93EC011B8E1A8E6DE10E944B0178
:100A3000482F4E7F6DE9CE01DF91CF910C94FF00DE
:100A4000CF93DF93EC0181E090E09B8F8A8F6DE183
:100A5000CE010E944B01482F41606DE9CE01DF912C
:100A6000CF910C94FF000F931F93CF93DF93EC0172
:100A70008B010E940903CE01012B99F00E942005F1
:100A800040E06DE8CE010E94FF0040E062EACE0146
:100A90000E94FF0081E090E0DF91CF911F910F91C4
:100AA00008950E941005ECCF0F931F93CF93DF930F
:100AB000EC018B011616170684F40E942005402FC6
:100AC00062EACE010E94FF0045E861E8CE01DF91B5
:100AD000CF911F910F910C94FF000E941005F4CF4D
:100AE0000F931F93CF93DF93EC0162E10E944B01C0
:100AF000182F482F62E9CE010E94FF0015FD25C086
:100B0000198E188E8A8D9B8D62E2892B09F463E120
:100B1000CE010E944B01082F10E060E1CE010E943F
:100B20004B01482F6DE8CE010E94FF00EC8DFD8D3A
:100B3000309711F0C801099540E06DE8CE01DF91D2
:100B4000CF911F910F910C94FF00DF91CF911F91D6
:100B50000F9108958AEA91E00C947005452B61F499
:100B6000AB016F30710514F04EE050E057FD40E0EE
:100B7000406769E80C94FF00AB016231710514F025
:100B800041E150E04230510514F442E050E042505F
:100B90004068EFCF8AEA91E00C94C8002F923F9210
:100BA0004F925F926F927F928F929F92AF92BF927D
:100BB000CF92DF92EF92FF920F931F93CF93DF9329
:100BC000CDB7DEB7C857D1090FB6F894DEBF0FBE58
:100BD000CDBFE9969FAF8EAFE9971A01DC01189659
:100BE0000D911D912D913C911B9761960CAF1DAFFE
:100BF0002EAF3FAF61971C960D911D912D913C91A9
:100C00001F9709831A832B833C8350960D911D9166
:100C10002D913C9153970D831E832F8338875496D3
:100C20000D911D912D913C91579709871A872B871C
:100C30003C87E6966FAFE697E7967FAFE797A85AAF
:100C4000BF4F6396BFAFAEAF6397FC01E45AFF4F4F
:100C50006596FFAFEEAF65978C01005A1F4F679600
:100C60001FAF0EAF67979C012C593F4F69963FAF5E
:100C70002EAF699788599F4F6B969FAF8EAF6B973A
:100C8000E996AEADBFADE997A459BF4F6D96BFAF22
:100C9000AEAF6D97E996EEADFFADE997E059FF4F26
:100CA0006F96FFAFEEAF6F97E9960EAD1FADE99768
:100CB0000C581F4FA1961FAF0EAFA197E9962EAD0E
:100CC0003FADE99728583F4FA3963FAF2EAFA3976C
:100CD000E9968EAD9FADE99784589F4FA5969FAF3B
:100CE0008EAFA597E996AEADBFADE997A058BF4FBF
:100CF000A796BFAFAEAFA797E996EEADFFADE99768
:100D0000EC57FF4FA996FFAFEEAFA997E9960EAD4E
:100D10001FADE99708571F4FAB961FAF0EAFAB97AC
:100D2000E9962EAD3FADE99724573F4FAD963FAFC3
:100D30002EAFAD97E9968EAD9FADE99780579F4F47
:100D4000AF969FAF8EAFAF97E996AEADBFADE997C7
:100D5000AC56BF4FE196BFAFAEAFE197E796AEADF1
:100D6000BFADE7970D911D912D913C910D871E8789
:100D70002F87388B6396EEADFFAD639700831183A9
:100D80002283338361968CAD9DADAEADBFAD6197CF
:100D900088589B45A549B842800F911FA21FB31FD9
:100DA0004D815E816F81788509851A852B853C850B
:100DB000402751276227732709811A812B813C81A3
:100DC000402351236223732309851A852B853C8593
:100DD0004027512762277327840F951FA61FB71F2F
:100DE0008C019D0147E0000F111F221F331F4A9500
:100DF000D1F7AC01BD01E9E1769567955795479527
:100E0000EA95D1F7402B512B622B732B89819A8164
:100E1000AB81BC81480F591F6A1F7B1FE796AEAD9F
:100E2000BFADE79714960D911D912D913C911797A9
:100E3000098B1A8B2B8B3C8B6596EEADFFAD6597BE
:100E4000008311832283338389859A85AB85BC8592
:100E50008A5A9844A843B741800F911FA21FB31F1D
:100E6000C980DA80EB80FC800D811E812F8138855E
:100E7000C026D126E226F326C422D522E622F72276
:100E8000C026D126E226F3268C0D9D1DAE1DBF1D6A
:100E90008C019D01FCE0000F111F221F331FFA95EA
:100EA000D1F76C017D01A4E1F694E794D794C7943F
:100EB000AA95D1F7C02AD12AE22AF32AC40ED51E58
:100EC000E61EF71EE796AEADBFADE79718968D917B
:100ED0009D910D90BC91A02D8D8B9E8BAF8BB88F6B
:100EE0006796EEADFFAD679780839183A283B3834E
:100EF0008D819E81AF81B88585529F48AF4DBB4D96
:100F00000D891E892F89388D800F911FA21FB31F55
:100F100049805A806B807C80442655266626772639
:100F20004C205D206E207F2009811A812B813C811D
:100F30004026512662267326840D951DA61DB71DD9
:100F40008C019D01EFE03695279517950795EA9559
:100F5000D1F72C013D01F1E1440C551C661C771CB6
:100F6000FA95D1F7402A512A622A732A4C0C5D1C4B
:100F70006E1C7F1CE796AEADBFADE7971C968D91BA
:100F80009D910D90BC91A02D898F9A8FAB8FBC8FB6
:100F90006996EEADFFAD699780839183A283B38399
:100FA00089819A81AB81BC8182519143A244BE4325
:100FB000098D1A8D2B8D3C8D800F911FA21FB31FA1
:100FC0008A019B010C251D252E253F250421152175
:100FD000262137210427152726273727800F911F21
:100FE000A21FB31F4C015D011AE0B694A794979419
:100FF00087941A95D1F78C019D0186E1000F111F8E
:10100000221F331F8A95D1F7082919292A293B293C
:10101000040D151D261D371DE796AEADBFADE79734
:1010200050968D919D910D90BC91A02D8D8F9E8F8E
:10103000AF8FB8A36B96EEADFFAD6B9780839183B6
:10104000A283B3838155904FA348BA40840F951F64
:10105000A61FB71FB701A60144255525662577258C
:1010600040235123622373234C255D256E257F2564
:10107000840F951FA61FB71F4C015D0147E0880C28
:10108000991CAA1CBB1C4A95D1F7AC01BD01E9E132
:101090007695679557954795EA95D1F74829592947
:1010A0006A297B29400F511F621F731FE796AEAD5F
:1010B000BFADE79754968D919D910D90BC91A02D59
:1010C00089A39AA3ABA3BCA36D96EEADFFAD6D97BC
:1010D00080839183A283B383865D9943A847B84BED
:1010E0008C0D9D1DAE1DBF1D73016201C026D12652
:1010F000E226F326C422D522E622F722C424D524F0
:10110000E624F7248C0D9D1DAE1DBF1D4C015D0115
:10111000FCE0880C991CAA1CBB1CFA95D1F76C0149
:101120007D01A4E1F694E794D794C794AA95D1F7EA
:10113000C828D928EA28FB28C40ED51EE61EF71EAB
:10114000E796AEADBFADE79758968D919D910D9006
:10115000BC91A02D8DA39EA3AFA3B8A76F96EEADB3
:10116000FFAD6F9780839183A283B3838D5E994B8C
:10117000AF4CB745840D951DA61DB71D280139013B
:1011800044265526662677264C205D206E207F203B
:101190004026512662267326840D951DA61DB71D77
:1011A0004C015D01EFE0B694A79497948794EA957B
:1011B000D1F72C013D01F1E1440C551C661C771C54
:1011C000FA95D1F7482859286A287B284C0C5D1CD1
:1011D0006E1C7F1CE796AEADBFADE7975C968D9118
:1011E0009D910D90BC91A02D89A79AA7ABA7BCA7F4
:1011F000A196EEADFFADA19780839183A283B383C7
:101200008F5F9A46A94BB240800F911FA21FB31F58
:101210008A019B010C251D252E253F250421152122
:10122000262137210427152726273727800F911FCE
:10123000A21FB31F4C015D011AE0B694A7949794C6
:1012400087941A95D1F78C019D0186E1000F111F3B
:10125000221F331F8A95D1F7082919292A293B29EA
:10126000040D151D261D371DE796AEADBFADE797E2
:1012700090968D919D910D90BC91A02D8DA79EA7CC
:10128000AFA7B8ABA396EEADFFADA39780839183D4
:10129000A283B38388529746AF47B649840F951F00
:1012A000A61FB71FB701A60144255525662577253A
:1012B00040235123622373234C255D256E257F2512
:1012C000840F951FA61FB71F4C015D0147E0880CD6
:1012D000991CAA1CBB1C4A95D1F7AC01BD01E9E1E0
:1012E0007695679557954795EA95D1F748295929F5
:1012F0006A297B29400F511F621F731FE796AEAD0D
:10130000BFADE79794968D919D910D90BC91A02DC6
:1013100089AB9AABABABBCABA596EEADFFADA597D9
:1013200080839183A283B38381559840AB4BB447AC
:101330008C0D9D1DAE1DBF1D73016201C026D126FF
:10134000E226F326C422D522E622F722C424D5249D
:10135000E624F7248C0D9D1DAE1DBF1D4C015D01C3
:10136000FCE0880C991CAA1CBB1CFA95D1F76C01F7
:101370007D01A4E1F694E794D794C794AA95D1F798
:10138000C828D928EA28FB28C40ED51EE61EF71E59
:10139000E796AEADBFADE79798968D919D910D9074
:1013A000BC91A02D8DAB9EABAFABB8AFA796EEAD09
:1013B000FFADA79780839183A283B3838F54944A10
:1013C000A109B109840D951DA61DB71D280139017C
:1013D00044265526662677264C205D206E207F20E9
:1013E0004026512662267326840D951DA61DB71D25
:1013F0004C015D01EFE0B694A79497948794EA9529
:10140000D1F72C013D01F1E1440C551C661C771C01
:10141000FA95D1F7482859286A287B284C0C5D1C7E
:101420006E1C7F1CE796AEADBFADE7979C968D9185
:101430009D910D90BC91A02D89AF9AAFABAFBCAF81
:10144000A996EEADFFADA99780839183A283B38364
:1014500082549842A34AB647800F911FA21FB31F20
:101460008A019B010C251D252E253F2504211521D0
:10147000262137210427152726273727800F911F7C
:10148000A21FB31F4C015D011AE0B694A794979474
:1014900087941A95D1F78C019D0186E1000F111FE9
:1014A000221F331F8A95D1F7082919292A293B2998
:1014B000040D151D261D371DE796AEADBFADE79790
:1014C000D0968D919D910D90BC91A02D21968CAFC1
:1014D0009DAFAEAFBFAF2197AB96EEADFFADAB9773
:1014E00080839183A283B3834C015D01FEED8F1A4B
:1014F000FEEE9F0AFFE6AF0AF4E9BF0A840E951ECE
:10150000A61EB71EB701A6014425552566257725D9
:1015100040235123622373234C255D256E257F25AF
:10152000480D591D6A1D7B1D4A015B0197E0880C1F
:10153000991CAA1CBB1C9A95D1F7E9E17695679591
:1015400057954795EA95D1F7482959296A297B2962
:10155000400F511F621F731FE796AEADBFADE797F7
:10156000D4968D919D910D90BC91A02D25968CAF18
:101570009DAFAEAFBFAF2597AD96EEADFFADAD97CA
:1015800080839183A283B3834C015D01FDE68F1AB2
:10159000FEE89F0AF7E6AF0AF2E0BF0A8C0C9D1C3A
:1015A000AE1CBF1C73016201C026D126E226F326C1
:1015B000C422D522E622F722C424D524E624F72427
:1015C000C80CD91CEA1CFB1C46015701FCE0880C26
:1015D000991CAA1CBB1CFA95D1F7A4E1F694E794D8
:1015E000D794C794AA95D1F7C828D928EA28FB2808
:1015F000C40ED51EE61EF71EE796AEADBFADE7974B
:10160000D8968D919D910D90BC91A02D29968CAF6F
:101610009DAFAEAFBFAF2997AF96EEADFFADAF9721
:1016200080839183A283B3834C015D01F2E78F1A1B
:10163000FCEB9F0AF6E8AF0AF9E5BF0A840C951C9B
:10164000A61CB71C28013901442655266626772694
:101650004C205D206E207F20402651266226732676
:10166000480C591C6A1C7B1C53014201BFE0B69414
:10167000A79497948794BA95D1F781E1440C551CAF
:10168000661C771C8A95D1F7482859286A287B2838
:101690004C0C5D1C6E1C7F1CE796AEADBFADE79792
:1016A000DC968D919D910D90BC91A02D2D968CAFC7
:1016B0009DAFAEAFBFAF2D97E196EEADFFADE19719
:1016C00080839183A283B3834C015D01FFED8F1A68
:1016D000F7EF9F0AFBE4AF0AF6EBBF0A800E911EFC
:1016E000A21EB31E8A019B010C251D252E253F2518
:1016F00004211521262137210427152726273727DE
:10170000080D191D2A1D3B1D480159019AE0B69488
:10171000A794979487949A95D1F7E6E1000F111F4B
:10172000221F331FEA95D1F7082919292A293B29B5
:10173000040D151D261D371D89889A88AB88BC8825
:101740008EE9881A8AED980A81EEA80A89E0B80A1B
:10175000840E951EA61EB71EB301A2014027512775
:10176000622773274C215D216E217F214425552559
:1017700066257725480D591D6A1D7B1D4A015B01B1
:10178000F5E0880C991CAA1CBB1CFA95D1F7ABE1BB
:101790007695679557954795AA95D1F74829592980
:1017A0006A297B29400F511F621F731F8DA09EA0C5
:1017B000AFA0B8A490EC891A9CE4990A9FEBA90AFF
:1017C0009FE3B90A8C0C9D1CAE1CBF1C68017901FB
:1017D000C426D526E626F726C420D520E620F72005
:1017E000C026D126E226F326C80CD91CEA1CFB1C15
:1017F00046015701B9E0880C991CAA1CBB1CBA957C
:10180000D1F787E1F694E794D794C7948A95D1F7F6
:10181000C828D928EA28FB28C40ED51EE61EF71EC4
:1018200089AC9AACABACBCACAFEA8A1AA5EA9A0A0E
:10183000A1EAAA0AA9EDBA0A840C951CA61CB71C39
:101840002A013B014C245D246E247F244022512236
:10185000622273224426552666267726480C591C98
:101860006A1C7B1C530142019EE0880C991CAA1C37
:10187000BB1C9A95D1F7E2E176946794579447940C
:10188000EA95D1F7482859286A287B284C0C5D1C1A
:101890006E1C7F1C8D849E84AF84B888B6E58B1A3D
:1018A000B8E39B0AB9E4AB0AB6E1BB0A800E911E0D
:1018B000A21EB31E9701860104251525262537256E
:1018C00004231523262337230C251D252E253F25EC
:1018D000080D191D2A1D3B1D48015901FCE0B69455
:1018E000A79497948794FA95D1F7A4E1000F111F5C
:1018F000221F331FAA95D1F7082919292A293B2924
:10190000040D151D261D371D89A09AA0ABA0BCA0F3
:10191000E3EA8E1AEFEE9E0AE0EDAE0AE9E2BE0AB5
:10192000840E951EA61EB71EB301A20140275127A3
:10193000622773274C215D216E217F214425552587
:1019400066257725480D591D6A1D7B1D4A015B01DF
:10195000B5E0880C991CAA1CBB1CBA95D1F78BE189
:1019600076956795579547958A95D1F748295929CE
:101970006A297B29400F511F621F731F8DA89EA8E3
:10198000AFA8B8ACFDEA8F1AFBEE9F0AFBEBAF0ADB
:10199000FDEFBF0A8C0C9D1CAE1CBF1C68017901B9
:1019A000C426D526E626F726C420D520E620F72033
:1019B000C026D126E226F326C80CD91CEA1CFB1C43
:1019C0004601570199E0880C991CAA1CBB1C9A95EA
:1019D000D1F7E7E1F694E794D794C794EA95D1F765
:1019E000C828D928EA28FB28C40ED51EE61EF71EF3
:1019F0002D968CAC9DACAEACBFAC2D978FE7881A02
:101A000089E1980A8EE5A80A87E2B80A840C951C39
:101A1000A61CB71C2A013B014C245D246E247F24A4
:101A200040225122622273224426552666267726BA
:101A3000480C591C6A1C7B1C53014201FEE0880CB7
:101A4000991CAA1CBB1CFA95D1F7A2E17694679465
:101A500057944794AA95D1F7482859286A287B2893
:101A60004C0C5D1C6E1C7F1C8D8C9E8CAF8CB8A0AA
:101A700098E3891A94E0990A9CE2A90A98E1B90AC4
:101A8000800E911EA21EB31E970186010425152506
:101A90002625372504231523262337230C251D252A
:101AA0002E253F25080D191D2A1D3B1D48015901F2
:101AB000BCE0B694A79497948794BA95D1F784E143
:101AC000000F111F221F331F8A95D1F708291929EA
:101AD0002A293B29040D151D261D371D89A89AA802
:101AE000ABA8BCA8AAE18A1AA2E39A0AAEE1AA0AA4
:101AF000AEEDBA0A840E951EA61EB71EB301A20152
:101B000040275127622773274C215D216E217F21B9
:101B10004425552566257725480D591D6A1D7B1DD1
:101B20004A015B0195E0880C991CAA1CBB1C9A9584
:101B3000D1F7EBE17695679557954795EA95D1F7FB
:101B4000482959296A297B29400F511F621F731F99
:101B500029968CAC9DACAEACBFAC2997BAE28B1A7F
:101B6000B8EF9B0AB8ECAB0ABCE3BB0A8C0C9D1C1B
:101B7000AE1CBF1C68017901C426D526E626F726CF
:101B8000C420D520E620F720C026D126E226F32661
:101B9000C80CD91CEA1CFB1C46015701F9E0880C53
:101BA000991CAA1CBB1CFA95D1F7A7E1F694E794FF
:101BB000D794C794AA95D1F7C828D928EA28FB2832
:101BC000C40ED51EE61EF71E898C9A8CAB8CBC8C7D
:101BD000E9E78E1AE2EF9E0AEAE2AE0AEBE0BE0AFD
:101BE000840C951CA61CB71C2A013B014C245D24C7
:101BF0006E247F24402251226222732244265526DD
:101C000066267726480C591C6A1C7B1C530142012E
:101C1000BEE0880C991CAA1CBB1CBA95D1F782E1C6
:101C200076946794579447948A95D1F74828592811
:101C30006A287B284C0C5D1C6E1C7F1C8DA49EA406
:101C4000AFA4B8A8F3E18F1AFBEE9F0AF5EAAF0A3A
:101C5000FAEBBF0A800E911EA21EB31E97018601E9
:101C60000425152526253725042315232623372368
:101C70000C251D252E253F25080D191D2A1D3B1D50
:101C8000480159019CE0B694A794979487949A953B
:101C9000D1F7E4E1000F111F221F331FEA95D1F79E
:101CA000082919292A293B29040D151D261D371D30
:101CB00025968CAC9DACAEACBFAC25978BEF881A4B
:101CC00086E1980A8CE1A80A86E5B80A840E951E7A
:101CD000A61EB71EB301A201402751276227732712
:101CE0004C215D216E217F214425552566257725D0
:101CF000480D591D6A1D7B1D4A015B01F5E0880CEA
:101D0000991CAA1CBB1CFA95D1F7ABE17695679597
:101D100057954795AA95D1F7482959296A297B29CA
:101D2000400F511F621F731F8D889E88AF88B88C2B
:101D300098E0891A9CE5990A90E1A90A93E0B90A0A
:101D40008C0C9D1CAE1CBF1C68017901C426D526D5
:101D5000E626F726C420D520E620F720C026D12687
:101D6000E226F326C80CD91CEA1CFB1C46015701CD
:101D7000B9E0880C991CAA1CBB1CBA95D1F787E165
:101D8000F694E794D794C7948A95D1F7C828D928B0
:101D9000EA28FB28C40ED51EE61EF71E89A49AA4C5
:101DA000ABA4BCA4A7E28A1AADEF9A0AA0E9AA0ADA
:101DB000A8E9BA0A840C951CA61CB71C2A013B0191
:101DC0004C245D246E247F244022512262227322FF
:101DD0004426552666267726480C591C6A1C7B1C0F
:101DE000530142019EE0880C991CAA1CBB1C9A95C9
:101DF000D1F7E2E17694679457944794EA95D1F746
:101E0000482859286A287B284C0C5D1C6E1C7F1CB6
:101E10004601570184249524A624B72421968CAD2D
:101E20009DADAEADBFAD21978657934BA54DB24743
:101E3000800F911FA21FB31F950184010423152356
:101E4000262337230C251D252E253F25800F911F86
:101E5000A21FB31F8C019D01FCE0369527951795B5
:101E60000795FA95D1F7E5960CAF1DAF2EAF3FAFB2
:101E7000E5978C019D01A4E1000F111F221F331F64
:101E8000AA95D1F7E5968CAD9DADAEADBFADE5970A
:101E9000082B192B2A2B3B2B040D151D261D371D36
:101EA00089A19AA1ABA1BCA18E5B964CA540B109BA
:101EB000840F951FA61FB71F80269126A226B32642
:101EC000880E991EAA1EBB1ED501C40144E0880FCE
:101ED000991FAA1FBB1F4A95D1F75CE1B694A7943E
:101EE000979487945A95D1F7882A992AAA2ABB2AC7
:101EF000800E911EA21EB31E4DA55EA56FA578A9EA
:101F00004F5759406E4878474C0D5D1D6E1D7F1D23
:101F100073016201C026D126E226F326C824D92403
:101F2000EA24FB24C40ED51EE61EF71EB701A60147
:101F3000EBE0440F551F661F771FEA95D1F7F5E1D7
:101F4000F694E794D794C794FA95D1F7C42AD52A82
:101F5000E62AF72AC80CD91CEA1CFB1C49AD5AAD6D
:101F60006BAD7CAD4E5D5E4962467249440E551EB6
:101F7000661E771EB901A801482559256A257B25CB
:101F80004C255D256E257F25440E551E661E771E49
:101F9000D20123013D014C0C5D1C6E1C7F1C299657
:101FA0004CAD5DAD6EAD7FAD2997445F574C6A4136
:101FB0007240400F511F621F731F950184010C2551
:101FC0001D252E253F250425152526253725040FFB
:101FD000151F261F371FB901A801A9E0769567953F
:101FE00057954795AA95D1F7B7E1000F111F221F0A
:101FF000331FBA95D1F7042B152B262B372B040D45
:10200000151D261D371D49895A896B897C894C5BB2
:10201000554161447B45480D591D6A1D7B1D460194
:10202000570184249524A624B72480269126A2262D
:10203000B326840E951EA61EB71EB501A40184E02A
:10204000440F551F661F771F8A95D1F79CE1B69400
:10205000A794979487949A95D1F7842A952AA62ACB
:10206000B72A800E911EA21EB31E4D8D5E8D6F8D00
:1020700078A1475550436142744BC40ED51EE61EED
:10208000F71EB301A2014027512762277327482575
:1020900059256A257B254C0D5D1D6E1D7F1DDB01BD
:1020A000CA01EBE0880F991FAA1FBB1FEA95D1F761
:1020B000F5E17695679557954795FA95D1F7482BB1
:1020C000592B6A2B7B2B480D591D6A1D7B1DC9A4FA
:1020D000DAA4EBA4FCA4B0EACB1AB4EBDB0AB4E4B8
:1020E000EB0AB9E0FB0A4C0C5D1C6E1C7F1C6801FE
:1020F0007901C824D924EA24FB24C426D526E6265F
:10210000F7264C0C5D1C6E1C7F1CF20123013F0165
:10211000440E551E661E771ECDA8DEA8EFA8F8ACAB
:10212000F0E9CF1AF3E4DF0AF0E4EF0AF1E4FF0A82
:10213000C00ED11EE21EF31E95018401042715274F
:102140002627372704251525262537250C0D1D1D87
:102150002E1D3F1D68017901A9E0F694E794D794FC
:10216000C794AA95D1F7B7E1000F111F221F331FA3
:10217000BA95D1F70C291D292E293F29040D151DCB
:10218000261D371D2596CCACDDACEEACFFAC2597FB
:102190008AE3C81A81E8D80A84E6E80A87EDF80AD3
:1021A000C80CD91CEA1CFB1C4A015B018424952441
:1021B000A624B72480269126A226B3268C0C9D1C2B
:1021C000AE1CBF1C7501640184E0CC0CDD1CEE1C50
:1021D000FF1C8A95D1F79CE1B694A79497948794B5
:1021E0009A95D1F78C289D28AE28BF28800E911E85
:1021F000A21EB31ECD84DE84EF84F88896E0C91A4F
:1022000098EDD90A9EE5E90A95E1F90AC40ED51EB2
:10221000E61EF71EB301A20140275127622773274C
:10222000482559256A257B254C0D5D1D6E1D7F1D9A
:102230006A017B01EBE0CC0CDD1CEE1CFF1CEA9577
:10224000D1F7F5E17695679557954795FA95D1F7CA
:102250004C295D296E297F29480D591D6A1D7B1D5A
:10226000C98CDA8CEB8CFC8CABE7CA1AAFECDA0ABF
:10227000A0E1EA0AABE2FA0A4C0C5D1C6E1C7F1C62
:1022800068017901C824D924EA24FB24C426D52670
:10229000E626F7264C0C5D1C6E1C7F1CF201230108
:1022A0003F01440E551E661E771ECDA0DEA0EFA096
:1022B000F8A4FBEFCF1AF2EEDF0AF7E7EF0AFBEF25
:1022C000FF0AC00ED11EE21EF31E950184010427F1
:1022D00015272627372704251525262537250C0DF4
:1022E0001D1D2E1D3F1D68017901A9E0F694E7949C
:1022F000D794C794AA95D1F7B7E1000F111F221FF9
:10230000331FBA95D1F70C291D292E293F29040D19
:10231000151D261D371DC9A8DAA8EBA8FCA887EC57
:10232000C81A8FE2D80A8BE2E80A86E2F80AC80CDB
:10233000D91CEA1CFB1C4A015B0184249524A624B9
:10234000B72480269126A226B3268C0C9D1CAE1C99
:10235000BF1C7501640184E0CC0CDD1CEE1CFF1C6D
:102360008A95D1F79CE1B694A794979487949A950F
:10237000D1F78C289D28AE28BF28800E911EA21E62
:10238000B31E2196CCACDDACEEACFFAC21979BE14B
:10239000C91A96E6D90A94E2E90A99E1F90AC40E43
:1023A000D51EE61EF71EB301A20140275127622762
:1023B0007327482559256A257B254C0D5D1D6E1D0B
:1023C0007F1D6A017B01EBE0CC0CDD1CEE1CFF1CC9
:1023D000EA95D1F7F5E17695679557954795FA9582
:1023E000D1F74C295D296E297F29480D591D6A1D99
:1023F0007B1D2D96CCACDDACEEACFFAC2D97A8E0F0
:10240000CA1AA3E8DA0AADE5EA0AA0EEFA0A4C0C09
:102410005D1C6E1C7F1C68017901C824D924EA2444
:10242000FB24C426D526E626F7264C0C5D1C6E1C24
:102430007F1CF20123013F01440E551E661E771ECC
:10244000CD88DE88EF88F88CFBE9CF1AF9EADF0A3D
:10245000F3E5EF0AFBE3FF0AC00ED11EE21EF31EF6
:1024600095018401042715272627372704251525DC
:10247000262537250C0D1D1D2E1D3F1D68017901D8
:10248000A9E0F694E794D794C794AA95D1F7B7E159
:10249000000F111F221F331FBA95D1F70C291D29D8
:1024A0002E293F29040D151D261D371DCD84DE84E0
:1024B000EF84F8888CEBC81A8DEDD80A86EDE80A0F
:1024C0008BE0F80AC80CD91CEA1CFB1C4A015B0112
:1024D00080949094A094B094802A912AA22AB32A3E
:1024E00084249524A624B7248C0C9D1CAE1CBF1CF0
:1024F0007501640186E0CC0CDD1CEE1CFF1C8A9586
:10250000D1F79AE1B694A794979487949A95D1F7C6
:102510008C289D28AE28BF28800E911EA21EB31EB7
:10252000C9A4DAA4EBA4FCA499E6C91AD10895EDD4
:10253000E90A9CEBF90AC40ED51EE61EF71EB3018C
:10254000A2014095509560957095482959296A29AE
:102550007B2940275127622773274C0D5D1D6E1D77
:102560007F1D6A017B01EAE0CC0CDD1CEE1CFF1C28
:10257000EA95D1F7F6E17695679557954795FA95DF
:10258000D1F74C295D296E297F29480D591D6A1DF7
:102590007B1D2996CCACDDACEEACFFAC2997A9E550
:1025A000CA1AACEDDA0AABE6EA0AA4E5FA0AC40CE8
:1025B000D51CE61CF71C2801390140945094609406
:1025C0007094442A552A662A772A482459246A2472
:1025D0007B244C0C5D1C6E1C7F1C73016201AFE000
:1025E000CC0CDD1CEE1CFF1CAA95D1F7B1E1769452
:1025F000679457944794BA95D1F74C285D286E2874
:102600007F28440E551E661E771EC9A0DAA0EBA0D7
:10261000FCA0B7ECCB1ABFE5DB0ABCE6EB0AB3E0E3
:10262000FB0AC00ED11EE21EF31E95018401009527
:102630001095209530950429152926293729042736
:102640001527262737270C0D1D1D2E1D3F1D680140
:1026500079018BE0F694E794D794C7948A95D1F7E3
:1026600095E1000F111F221F331F9A95D1F70C29F6
:102670001D292E293F29040D151D261D371D2196C4
:10268000CCACDDACEEACFFAC2197EDE3CE1AE6EAC4
:10269000DE0AE4EAEE0AEAE9FE0AC80CD91CEA1CE2
:1026A000FB1C4A015B0180949094A094B094802A12
:1026B000912AA22AB32A84249524A624B7248C0C18
:1026C0009D1CAE1CBF1C75016401E6E0CC0CDD1C3A
:1026D000EE1CFF1CEA95D1F7FAE1B694A794979403
:1026E0008794FA95D1F78C289D28AE28BF28800EB4
:1026F000911EA21EB31EC98CDA8CEB8CFC8CFEE6FC
:10270000CF1AF3E3DF0AF3EFEF0AF0E7FF0AC40E94
:10271000D51EE61EF71EB301A201409550956095A7
:102720007095482959296A297B2940275127622712
:1027300073274C0D5D1D6E1D7F1D6A017B01AAE094
:10274000CC0CDD1CEE1CFF1CAA95D1F7B6E17695EA
:10275000679557954795BA95D1F74C295D296E290C
:102760007F29480D591D6A1D7B1DCDA8DEA8EFA845
:10277000F8AC83E8C81A8BE0D80A80E1E80AF108CF
:10278000C40CD51CE61CF71C280139014094509458
:1027900060947094442A552A662A772A482459243A
:1027A0006A247B244C0C5D1C6E1C7F1C730162012F
:1027B0008FE0CC0CDD1CEE1CFF1C8A95D1F791E15B
:1027C00076946794579447949A95D1F74C285D284E
:1027D0006E287F28440E551E661E771EC988DA882B
:1027E000EB88FC889FE2C91A92EAD90A9BE7E90ABA
:1027F0009AE7F90AC00ED11EE21EF31E950184016C
:1028000000951095209530950429152926293729FA
:1028100004271527262737270C0D1D1D2E1D3F1DAC
:1028200068017901EBE0F694E794D794C794EA95B0
:10283000D1F7F5E1000F111F221F331FFA95D1F7D1
:102840000C291D292E293F29040D151D261D371D74
:10285000CDA4DEA4EFA4F8A8A1EBCA1AA1E8DA0A75
:10286000A7E5EA0AA0E9FA0AC80CD91CEA1CFB1C75
:102870004A015B0180949094A094B094802A912A9C
:10288000A22AB32A84249524A624B7248C0C9D1C48
:10289000AE1CBF1C75016401A6E0CC0CDD1CEE1C57
:1028A000FF1CAA95D1F7BAE1B694A79497948794A0
:1028B000BA95D1F78C289D28AE28BF28800E911E8E
:1028C000A21EB31E2D968CAD9DADAEADBFAD2D97A6
:1028D00080529941A34DB140840F951FA61FB71F89
:1028E000B301A201409550956095709548295929EA
:1028F0006A297B294027512762277327840F951F58
:10290000A61FB71F6C017D014AE0CC0CDD1CEE1C3C
:10291000FF1C4A95D1F7AC01BD01E6E176956795BC
:1029200057954795EA95D1F74C295D296E297F295E
:10293000480D591D6A1D7B1D8DA19EA1AFA1B8A593
:102940008C5E9C4BAE4FBC45840D951DA61DB71DDE
:10295000280139014094509460947094442A552A77
:10296000662A772A482459246A247B24840D951DDD
:10297000A61DB71D6C017D01FFE0CC0CDD1CEE1C1B
:10298000FF1CFA95D1F72C013D01A1E176946794E3
:1029900057944794AA95D1F74C285D286E287F2834
:1029A000440E551E661E771E25968CAD9DADAEADB0
:1029B000BFAD25978F559E4EA74FB14B800F911FEE
:1029C000A21FB31F950184010095109520953095A5
:1029D00004291529262937290427152726273727CB
:1029E000800F911FA21FB31F6C017D011BE0F694A5
:1029F000E794D794C7941A95D1F78C019D0185E18E
:102A0000000F111F221F331F8A95D1F70C291D2992
:102A10002E293F29040D151D261D371D8D8D9E8DD8
:102A2000AF8DB8A18E579148AC4AB840880D991D1A
:102A3000AA1DBB1D4A015B0180949094A094B094A0
:102A4000802A912AA22AB32A84249524A624B72472
:102A5000880D991DAA1DBB1D6C017D01E6E0CC0C03
:102A6000DD1CEE1CFF1CEA95D1F74C015D01FAE17B
:102A7000B694A79497948794FA95D1F78C289D28BB
:102A8000AE28BF28800E911EA21EB31E89AD9AAD3E
:102A9000ABADBCAD8B5C9D40A54CB244840F951F83
:102AA000A61FB71FB301A201409550956095709580
:102AB000482959296A297B294027512762277327EA
:102AC000840F951FA61FB71F6C017D014AE0CC0C37
:102AD000DD1CEE1CFF1C4A95D1F7AC01BD01E6E1FF
:102AE0007695679557954795EA95D1F74C295D29D5
:102AF0006E297F29480D591D6A1D7B1D8D899E8970
:102B0000AF89B88D85549D42A842B54D840D951D61
:102B1000A61DB71D2801390140945094609470940B
:102B2000442A552A662A772A482459246A247B2471
:102B3000840D951DA61DB71D6C017D01FFE0CC0C19
:102B4000DD1CEE1CFF1CFA95D1F72C013D01A1E123
:102B50007694679457944794AA95D1F74C285D28AA
:102B60006E287F28440E551E661E771E89A99AA9D5
:102B7000ABA9BCA98F569C42A947B441800F911FB5
:102B8000A21FB31F950184010095109520953095E3
:102B90000429152926293729042715272627372709
:102BA000800F911FA21FB31F6C017D011BE0F694E3
:102BB000E794D794C7941A95D1F78C019D0185E1CC
:102BC000000F111F221F331F8A95D1F70C291D29D1
:102BD0002E293F29040D151D261D371D61968CAD2C
:102BE0009DADAEADBFAD6197880D991DAA1DBB1DF2
:102BF00061968CAF9DAFAEAFBFAF619789819A816F
:102C0000AB81BC81800F911FA21FB31F89839A8360
:102C1000AB83BC830D811E812F813885040D151D6A
:102C2000261D371D0D831E832F83388789859A853E
:102C3000AB85BC85840F951FA61FB71F89879A8710
:102C4000AB87BC87E796AEADBFADE797A05CBF4F43
:102C5000E796BFAFAEAFE797B0E42B1A310811F09B
:102C60000C94AE0661960CAD1DAD2EAD3FAD6197D7
:102C7000E996AEADBFADE99718960D931D932D93D0
:102C80003C931B9709811A812B813C811C960D93E3
:102C90001D932D933C931F970D811E812F813885A5
:102CA00050960D931D932D933C93539709851A8548
:102CB0002B853C8554960D931D932D933C935797EC
:102CC000E7968EAD9FADE797C858DF4F0FB6F894E3
:102CD000DEBF0FBECDBFDF91CF911F910F91FF904F
:102CE000EF90DF90CF90BF90AF909F908F907F90AC
:102CF0006F905F904F903F902F900895CF93DF9308
:102D0000FC0181E093E2A5E4B7E680879187A28782
:102D1000B38789E89BEAADECBFEE84879587A687E9
:102D2000B7878EEF9CEDAAEBB8E9808B918BA28BD5
:102D3000B38B86E794E5A2E3B0E1848B958BA68BF9
:102D4000B78B10821182128213821482158216822E
:102D50001782DF01A85ABF4F80E4ED01982F199226
:102D60009A95E9F77896DF011D928A95E9F7DF9148
:102D7000CF9108958F929F92AF92BF92EF92FF9260
:102D80000F931F93CF93DF93EC017B018A0188811E
:102D90009981AA81BB8170E060E04A015B01880EE5
:102DA000991EAA1EBB1E2FE1B22288829982AA8296
:102DB000BB8288169906AA06BB0668F48C809D80A3
:102DC000AE80BF802FEF821A920AA20AB20A8C82CA
:102DD0009D82AE82BF828F739927AA27BB27009757
:102DE000A105B10579F120E4822E912CA12CB12C02
:102DF000881A990AAA0ABB0A48968C0F9D1F481583
:102E000059056A057B0570F4A801B701DF91CF91E0
:102E10001F910F91FF90EF90BF90AF909F908F9078
:102E20000C940530A401B7010E940530E80CF91C90
:102E30000819190940E450E0BE01685E7F4FCE01D9
:102E40000E94CE050034110548F0A801407CB7016E
:102E5000CE010E94CE057C010F731127A801B70196
:102E6000CE014896D3CFEF92FF920F931F93CF934B
:102E7000DF938C01EB01488159816A817B814F731B
:102E8000552766277727DB01CA010196A11DB11DD1
:102E90004C0F5D1F20E8FA01208F40E450E060E015
:102EA00070E0481B590B6A0B7B0B7E01F8E1EF0EBB
:102EB000F11C4830510561057105A0F4489670E099
:102EC00060E08C0F9D1F0E940E3040E450E0B7017F
:102ED000CE010E94CE0540E450E060E070E080E06A
:102EE00090E0DC0148505109489670E060E08C0F9A
:102EF0009D1F0E940E3088819981AA81BB8123E0A9
:102F0000880F991FAA1FBB1F2A95D1F78883998321
:102F1000AA83BB83FE01E05BFF4F808331969083E1
:102F20003196A0833196B0833C812D819E818F8123
:102F30003196308331962083319690833196808309
:102F400040E450E0B701CE010E94CE058885F8012B
:102F50008083898581838A8582838B8583838C8521
:102F600084838D8585838E8586838F8587838889F5
:102F70008087898981878A8982878B8983878C89E1
:102F800084878D8985878E8986878F89878788E959
:102F9000FE0111928A95E9F7DF91CF911F910F9170
:102FA000FF90EF900895CF92DF92EF92FF920F93F0
:102FB0001F93CF93DF93CDB7DEB7C859D1090FB6B2
:102FC000F894DEBF0FBECDBF7C016B0180E190E0C5
:102FD0000E9436278C01CE0101960E947E16A60122
:102FE000B701CE0101960E94BA16BE016F5F7F4FF6
:102FF000C8010E943317C801C856DF4F0FB6F894B6
:10300000DEBF0FBECDBFDF91CF911F910F91FF901B
:10301000EF90DF90CF9008951F93CF93DF93EC0153
:10302000162F0E941530181739F0612FCE01DF914D
:10303000CF911F910C941D30DF91CF911F91089576
:103040000C941530DC01ED91FC910190F081E02DA4
:10305000099461E08CE00C94622A60E08CE00C94AE
:10306000622A61E08DE00C94622A60E08DE00C94AD
:10307000622A88E198E00FB6F894A89580936000E2
:103080000FBE909360000E9431180E942D18FBCF54
:103090000F931F93CF93DF938C01EC01892B11F4D5
:1030A000C1E0D0E01C161D060CF561E08CE00E942A
:1030B000622A60E08DE00E94622A64E670E080E0AF
:1030C00090E00E94D72860E08CE00E94622A61E0D4
:1030D0008DE00E94622A64E670E080E090E00E9449
:1030E000D72801151105F1F22197DCCF0E942D1888
:1030F000DF91CF911F910F910C9435180E943118D8
:103100000E942D186AE070E080E090E00E94D728CD
:103110000E9429180E94351865E070E080E090E078
:103120000E94D728EBCF0F931F93CF93DF938C018F
:10313000EC01892B11F4C1E0D0E061E08DE00E9448
:10314000622A1C161D06ACF40E94351864E670E075
:1031500080E090E00E94D7280E94311864E670E079
:1031600080E090E00E94D7280115110551F32197C6
:10317000E8CFDF91CF911F910F910C9435180F93E9
:103180001F93CF93DF938C01EC01892B11F4C1E0E5
:10319000D0E01C161D06ACF40E942D1864E670E009
:1031A00080E090E00E94D7280E94291864E670E031
:1031B00080E090E00E94D7280115110551F3219776
:1031C000E8CFDF91CF911F910F910C942D18809132
:1031D000113590911235A0911335B09114350196A7
:1031E000A11DB11D8093113590931235A093133515
:1031F000B09314354091040150910501609106018E
:1032000070910701481759076A077B0710F510925C
:1032100011351092123510921335109214356091B9
:10322000103580910901861770F081E080930F3589
:1032300080910F35680F6093103570E08CE00E942C
:1032400076290C94351880910801681788F38FEF60
:10325000EDCF08958091113590911235A0911335DD
:10326000B09114350196A11DB11D80931135909335
:103270001235A0931335B093143540910401509149
:1032800005016091060170910701481759076A0707
:103290007B0710F5109211351092123510921335EC
:1032A000109214356091103580910901861770F0E5
:1032B00081E080930F3580910F35680F6093103552
:1032C00070E08DE00E9476290C942D188091080101
:1032D000681788F38FEFEDCF089560EC70E08BE313
:1032E00099E30E94221866E070E08BE399E30E9464
:1032F00022186091233970E08BE399E30E94221831
:1033000060EC70E08BE399E30C94221860EC70E0C1
:103310008BE399E30E94221867E070E08BE399E366
:103320000E9422186091150170E08BE399E30E94DE
:10333000221860EC70E08BE399E30C94221860ECA7
:1033400070E08BE399E30E9422186FE070E08BE35A
:1033500099E30E94221861E070E08BE399E30E94F8
:10336000221860EC70E08BE399E30C94221860EC77
:1033700070E08BE399E30E9422186FE070E08BE32A
:1033800099E30E94221870E060E08BE399E30E94C9
:10339000221860EC70E08BE399E30C94221860EC47
:1033A00070E08BE399E30E9422186EE070E08BE3FB
:1033B00099E30E9422188091213961E070E0811127
:1033C00002C070E060E08BE399E30E94221860EC99
:1033D00070E08BE399E30C94221860EC70E08BE3CF
:1033E00099E30E94221868E070E08BE399E30E9461
:1033F000221866E470E08BE399E30E94221860ECE7
:1034000070E08BE399E30C94221860EC70E08BE39E
:1034100099E30E94221860E570E08BE399E30E9433
:10342000221861E070E08BE399E30E9422186AE1C0
:1034300070E08BE399E30E94221860EC70E08BE36C
:1034400099E30C94221860EC70E08BE399E30E94FE
:10345000221868E470E08BE399E30E94221860E987
:1034600070E08BE399E30E94221860EC70E08BE33C
:1034700099E30C94221860EC70E08BE399E30E94CE
:10348000221867E470E08BE399E30E94221861E35D
:1034900070E08BE399E30E94221860EC70E08BE30C
:1034A00099E30C94221860EC70E08BE399E30E949E
:1034B000221869E470E08BE399E30E94221861E925
:1034C00070E08BE399E30E94221860EC70E08BE3DC
:1034D00099E30C94221880912339882341F060915C
:1034E0002C3970912D398AEA91E00C9407040895E3
:1034F00080912339882341F060911801709119015E
:103500008AEA91E00C94E004089580931F3988239F
:1035100021F081E080932039089510922039089598
:10352000809123398823E1F080911E39843A51F447
:10353000609116017091170150E040E08AEA91E035
:103540000E94AE0580911E39893A51F460911601AE
:103550007091170141E050E08AEA91E00C94AE05C9
:10356000089580912339882361F08AEA91E00E94CE
:103570000A02609328397093293980932A399093ED
:103580002B39089580912339882371F0409128398F
:103590005091293960912A3970912B398AEA91E04A
:1035A0000E9446040C94B11A08958091233988230F
:1035B00061F08AEA91E00E94DA0160932439709305
:1035C000253980932639909327390895809123399E
:1035D000882371F040912439509125396091263922
:1035E000709127398AEA91E00E9415030C94D51A4C
:1035F000089580912339882321F08AEA91E00C9480
:10360000280280E0089583ED9FE00E94201891E059
:10361000833709F090E0892F0895C8E3DFE06FEF6A
:10362000CE010E940C182196C11580E1D807B9F788
:103630000E94391888E39FE00E942018982F81E0AB
:10364000933021F0903F11F080E00895089589E3D0
:103650009FE00E942018982F80931E3981E0943AB1
:1036600021F0993A11F080E0089508958AE39FE0EF
:103670000E94201880931D399FEF980F81E09E3F94
:1036800008F080E00895BF92CF92DF92EF92FF9210
:103690000F931F93CF93DF938BE090E00E94362728
:1036A0007C018C01C8E3DFE0CE010E942018F80104
:1036B00081938F012196C334FFE0DF07A9F76BE008
:1036C00070E0C7010E94D317B82EC92E082F192FFA
:1036D000DD24D394CE010E942018F80191918F012E
:1036E0008913D12C2196C335FFE0DF0799F78B2D85
:1036F0009C2D0E94D227C7010E94D2278D2DDF91D9
:10370000CF911F910F91FF90EF90DF90CF90BF90DE
:1037100008958FED9FE00E94201891E0833709F013
:1037200090E0892F0895CF92DF92EF92FF92CF938E
:103730000E94891B882309F461C084ED9FE00E94E8
:10374000201890E090932D3980932C3985ED9FE0DF
:103750000E94201890E0909319018093180186ED43
:103760009FE00E94201890E090931701809316012B
:103770008BED9FE00E942018C82F8CED9FE00E94E7
:10378000201890E0B0E0A0E07C01DD24CC24FC2AED
:103790008DED9FE00E942018C82F8EED9FE00E94C3
:1037A0002018C82ADC2AC0922439D0922539E09208
:1037B0002639F092273987ED9FE00E942018C82F04
:1037C00088ED9FE00E94201890E0B0E0A0E07C012E
:1037D000DD24CC24FC2A89ED9FE00E942018C82F0C
:1037E0008AED9FE00E942018C82ADC2AC09228395E
:1037F000D0922939E0922A39F0922B39CF91FF905B
:10380000EF90DF90CF90089580912239882309F4BA
:103810008AC080912339882309F485C060912C39AE
:1038200084ED9FE00E940C186091180185ED9FE0E7
:103830000E940C186091160186ED9FE00E940C1802
:10384000609128397091293980912A3990912B39CA
:10385000692F77278827992787ED9FE00E940C180A
:10386000609128397091293980912A3990912B39AA
:10387000BC018827992788ED9FE00E940C18609171
:1038800028397091293980912A3990912B39672FE5
:10389000782F892F992789ED9FE00E940C1860915D
:1038A00028398AED9FE00E940C18609124397091AC
:1038B00025398091263990912739692F77278827D4
:1038C00099278BED9FE00E940C186091243970912C
:1038D00025398091263990912739BC01882799276D
:1038E0008CED9FE00E940C1860912439709125396D
:1038F0008091263990912739672F782F892F992722
:103900008DED9FE00E940C18609124398EED9FE0B0
:103910000E940C1863E78FED9FE00E940C188AE06C
:1039200090E00C94BF188AE090E00C94931860E04B
:103930008FED9FE00C940C1882E390E00E944818F1
:103940000E940D1B8091203970E060E0882319F0FF
:1039500060911F3970E08AEA91E00C9454058AEA7C
:1039600091E00E9411031092233908958091243927
:1039700090912539A0912639B0912739892B8A2B2E
:103980008B2BE1F08091283990912939A0912A3927
:10399000B0912B39892B8A2B8B2B81F080911601CA
:1039A000909117018F3F910549F080912C399091AA
:1039B0002D39892B19F010921501089581E080931B
:1039C000150108958091D101883C50F42091CF01D8
:1039D0003091D00181E02115384118F480E008953C
:1039E00081E00895CF938AEA91E00E944F01C82FA9
:1039F0000E94A62860931A3570931B3580931C355E
:103A000090931D35C0FF2DC081E0809325358093B4
:103A100024358093233580911E3590911F35209158
:103A20002535211108C020912435211104C0209191
:103A30002335222319F120910F01309110018217B3
:103A40009307B0F4019690931F3580931E3581E063
:103A500080932235809121358823E9F0CF910C9411
:103A60002918109225351092243510922335D3CF82
:103A700081E08093223580932135ECCF009741F08F
:103A8000019790931F3580931E3510922235E2CF17
:103A900010922135FACFCF910C942D180F931F93CC
:103AA0000E94A62800911A3510911B3520911C35D3
:103AB00030911D35601B710B820B930B00910B0134
:103AC00010910C0120910D0130910E0160177107CA
:103AD0008207930720F01F910F910C94F21C1F9105
:103AE0000F9108951092900089E18093910080E8F1
:103AF0009EE3909397008093960080E280937100FC
:103B0000089580910901809310350895803C61F4F7
:103B10006BED70E08BE399E30E9422188CED682F27
:103B20008BE399E30C941A2B8B3DC9F76BED70E096
:103B30008BE399E30E9422188DEDF1CF60EC70E0E9
:103B40008BE399E30E94221861E270E08BE399E332
:103B50000E94221880912D350E94861D80912C355F
:103B60000E94861D80912B350E94861D80912A35EA
:103B70000E94861D60EC70E08BE399E30C942218A0
:103B800060EC70E08BE399E30E94221862E270E03F
:103B90008BE399E30E942218809129350E94861DAB
:103BA000809128350E94861D809127350E94861DB0
:103BB000809126350E94861D60EC70E08BE399E3CE
:103BC0000C942218CF93C0911201C35660EC70E0A0
:103BD0008BE399E30E94221863E270E08BE399E3A0
:103BE0000E9422188C2F0E94861D60EC70E08BE3EF
:103BF00099E3CF910C94221860EC70E08BE399E389
:103C00000E94221864E270E08BE399E30E9422187C
:103C100080911C390E94861D60EC70E08BE399E373
:103C20000C94221860EC70E08BE399E30E94221858
:103C300062E070E08BE399E30E94221880912B39B7
:103C40000E94861D80912A390E94861D8091293903
:103C50000E94861D809128390E94861D60EC70E0CC
:103C60008BE399E30C94221860EC70E08BE399E30A
:103C70000E94221861E070E08BE399E30E94221811
:103C8000809127390E94861D809126390E94861DC9
:103C9000809125390E94861D809124390E94861DBD
:103CA00060EC70E08BE399E30C942218CF93DF93E0
:103CB000C8E3DFE0CE010E9420180E94861D2196F5
:103CC000C11580E1D807B1F7DF91CF91089560EC7D
:103CD00070E08BE399E30E94221861E570E08BE3CA
:103CE00099E30E9422180E94561E60EC70E08BE35C
:103CF00099E30C942218CF93C82F60EC70E08BE30B
:103D000099E30E94221860E970E08BE399E30E9436
:103D100022186C2F8BE399E30E941A2B60EC70E061
:103D20008BE399E3CF910C942218CF93DF93C82FA4
:103D3000D62F0E94031B81110BC0C83C48F48C2F66
:103D400090E06D2F885C904FDF91CF910C940C1810
:103D500083E0DF91CF910C947B1ECF93DF930E9481
:103D6000B61CC0912339C11149C080911501811140
:103D70003EC0D0912239DD23D1F1409124395091B8
:103D8000253960912639709127398AEA91E00E949D
:103D90006403892B59F481E00E947B1E90E080E04F
:103DA0000E9448188C2FDF91CF91089581E0809375
:103DB00023390E94901A0E94C21A0E946B1A0E9414
:103DC000781A0E94D51A8AEA91E00E94020568EAF0
:103DD00072E28AEA91E00E94A6020E94A21C0E945E
:103DE0006D1983E090E00E94BF18CD2FDBCF0E94B9
:103DF0006D1983E090E00E949318D4CF0E946D1952
:103E0000D1CF60EC70E08BE399E30E94221864E06C
:103E100070E08BE399E30E94221860912C398BE3C8
:103E200099E30E941A2B60EC70E08BE399E30C9409
:103E3000221860EC70E08BE399E30E94221865E0A1
:103E400070E08BE399E30E942218609118018BE3E4
:103E500099E30E941A2B60EC70E08BE399E30C94D9
:103E6000221860EC70E08BE399E30E94221869E06D
:103E700070E08BE399E30E94221860911F398BE375
:103E800099E30E941A2B60EC70E08BE399E30C94A9
:103E9000221860EC70E08BE399E30E94221863E043
:103EA00070E08BE399E30E942218609116018BE386
:103EB00099E30E941A2B60EC70E08BE399E30C9479
:103EC0002218CF93C82F60EC70E08BE399E30E9437
:103ED000221860E470E08BE399E30E9422186C2FB3
:103EE0008BE399E30E941A2B60EC70E08BE399E37B
:103EF000CF910C94221890911735992309F48EC212
:103F0000803C09F0ACC080910A0181119DC01092E3
:103F100017358091021D9091031D6091FE1C7091D8
:103F2000FF1C8617970761F42091041D3091051D31
:103F30008091001D9091011D2817390709F471C265
:103F40002091041D3091051D8091021D9091031D4B
:103F500002972817390709F464C28091CF01909124
:103F6000D0018115984108F05CC22091CB013091BD
:103F7000CC018091CD019091CE01019710F48FEF8B
:103F800097E18217930709F44BC02817390708F007
:103F900042C0821B930B0196009709F442C24091E4
:103FA000D1014F5F4093D101E091041DF091051DB7
:103FB000318320834091041D5091051D2091001DE7
:103FC0003091011D4217530771F57093051D6093E1
:103FD000041DE0916A1BF0916B1B918380832091FB
:103FE0006A1B30916B1B8091661B9091671B281791
:103FF000390721F58091641B9091651B90936B1B91
:1040000080936A1B8091CD019091CE019093CC0159
:104010008093CB010895821B930B8F5F974EBCCF8B
:1040200081E090E0BCCF2091041D3091051D2E5FF2
:104030003F4F3093051D2093041DCBCF80916A1B09
:1040400090916B1B0296DACF81E0809317358EEF4B
:1040500080930A0110921935109218350895209115
:10406000183530911935243F91E0390708F0D9C14E
:1040700090910A012115310529F49E3F19F480938E
:104080000A010895911146C08B3D21F481E080938F
:104090001635089590911635992349F08C3D21F0FD
:1040A0008D3D19F48BED01C080EC10921635909186
:1040B000D101983C08F0B5C12091CF013091D001D9
:1040C0002115384108F0ADC12091CF013091D001C8
:1040D0002F5F3F4F3093D0012093CF012091CD012E
:1040E0003091CE01A9014F5F5F4F5093CE014093B5
:1040F000CD012E523E4FF90180838091CD019091E8
:10410000CE018115984109F08CC11092CE01109218
:10411000CD010895913009F044C08B3DD1F49093C6
:1041200016358091183590911935049709F079C1A9
:1041300060912237709123378091243790912537F1
:104140000E94772E6115710581059105D9F40C94B3
:10415000341E90911635992349F08C3D21F08D3D08
:1041600019F48BED01C080EC10921635A9014F5F58
:104170005F4F50931935409318352E5D384CF90137
:104180008083CFCF6093243970932539809326396B
:1041900090932739809114018131C9F60E94E61A63
:1041A000D6CF923009F045C08B3DD9F481E08093A1
:1041B00016358091183590911935049709F031C161
:1041C0006091223770912337809124379091253761
:1041D0000E94772E6115710581059105D9F40C9423
:1041E000121E90911635992349F08C3D21F08D3D9A
:1041F00019F48BED01C080EC10921635A9014F5FC8
:104200005F4F50931935409318352E5D384CF901A6
:104210008083CFCF609328397093293980932A39CE
:1042200090932B39809114018131C9F60E94C21AF2
:10423000D6CF933099F48F3F11F40C94491F8231FB
:1042400008F081E190E0909317018093160180912E
:104250001401813191F70E94901AEFCF9430D1F47C
:104260008F3F11F40C94011F863088F090E08D3060
:10427000910514F08CE090E090932D3980932C39C7
:1042800080911401813171F70E946B1AEBCF86E0A7
:1042900090E0F2CF9530D1F48F3F11F40C94191FB8
:1042A000853088F090E08930910514F088E090E046
:1042B000909319018093180180911401813171F755
:1042C0000E94781AEBCF85E090E0F2CF993021F48C
:1042D0000E94851A0C94311F963079F48F3F11F4A7
:1042E0000C946D19811103C00E94AF1CF9CF81306D
:1042F00009F097C00E94AD1EF3CF913211F40C94D7
:104300009E1D923211F40C94C01D933211F40C9442
:10431000E21D973021F40E94B61C0C94861990334C
:1043200019F490E00C94BF18903421F40E94F91A0B
:104330000C94611F983029F4833709F072C00C94F3
:10434000ED199E3059F4813021F4809321390C9479
:10435000CF198111FCCF10922139F9CF9F3041F450
:104360000E94E21C811102C00C949F190C94B71991
:10437000993529F4883F09F054C00E949C1C95355A
:1043800029F4883F09F04DC00E943918913511F485
:104390000C94671E923551F58B3D79F481E0809342
:1043A000163580911835909119350297D1F56091A5
:1043B0002337809122370C94951E909116359923BE
:1043C00049F08C3D21F08D3D19F48BED01C080EC5E
:1043D00010921635A9014F5F5F4F509319354093E6
:1043E00018352E5D384CF9018083DBCF903511F400
:1043F0000C94051A983411F40C94231A993411F47E
:104400000C94531A973411F40C943B1A933511F40D
:104410000C94041C943529F40C94971C803C09F4EA
:1044200013CE089581E08093C8014FB7F89420918E
:104430000B3530910C3580910D3590910E354FBF75
:1044400028173907F1F0E0910B35F0910C35809188
:10445000093590910A35E817F90761F4809107351D
:104460009091083590930C3580930B3580810E9494
:104470007B1FDBCFE0910B35F0910C35CF0101961E
:10448000F1CF1092C8010895CF93DF9360EC70E0F4
:104490008BE399E30E94221870E060E08BE399E3DC
:1044A0000E942218C6E2D7E320911A3930911B39B5
:1044B000CE018652974382179307C8F46991603CF6
:1044C00061F46BED70E08BE399E30E9422186CEDD0
:1044D0008BE399E30E941A2BE7CF6B3DC9F76BED95
:1044E00070E08BE399E30E9422186DEDF1CF60EC50
:1044F00070E08BE399E30E94221810921B3910920E
:104500001A39DF91CF910895CF93DF93EC01209773
:10451000E1F0219780911A3990911B39843F9140A5
:10452000A0F48AEA91E00E94BF0120911A393091EB
:104530001B39A9014F5F5F4F50931B3940931A39C4
:104540002A5D384CF9018083E2CFDF91CF91089545
:104550000F931F93CF93DF93EC0180912139811149
:104560007BC08AEA91E00E94BF012197409111012E
:1045700080FF57C09C0154E0359527955A95E1F787
:104580002F7033274F3FD9F410921B3910921A39EC
:10459000209311018AEA91E00E9466019093130131
:1045A000809312018AEA91E00E94520180931C39A3
:1045B000CE01DF91CF911F910F910C94842224138F
:1045C000E3CF8AEA91E00E946601209112013091C6
:1045D0001301820F931F97FD0196959587959093F0
:1045E00013018093120100911C3910E08AEA91E0D6
:1045F0000E945201800F912F911D95958795809370
:104600001C39CE010E9484228FEF809311010E94F9
:10461000E21D0E94FC1DDF91CF911F910F910C9420
:1046200044224F3F39F010921B3910921A398FEF04
:10463000809311018AEA91E00E9466019093130130
:10464000809312018AEA91E00E94520180931C3902
:10465000CE010E948422DBCF10921B3910921A39AE
:10466000E9CFCF92DF92EF92FF920F931F93CF93F8
:10467000DF93EC0180912339882309F479C080917C
:104680002139811153C00E94311860E071E080E04F
:1046900090E00E94952C162F107FCF3FD10508F097
:1046A000116070E060E08AEA91E00E943305612FBA
:1046B0008AEA91E00E94B1009EE2C92E95E3D92ECC
:1046C000C25DDA4CEE24E394F12CCC16DD06F1F059
:1046D000F60161916F018AEA91E00E94B100FFEF5B
:1046E000EF1AFF0A8FEFE816F10479F78AEA91E0F2
:1046F0000E942B0270E060E08AEA91E00E9433059C
:10470000612F8AEA91E00E94B100DCCF8AEA91E051
:104710000E942B020E943518DF91CF911F910F91BB
:10472000FF90EF90DF90CF900C94A21C0E94311864
:10473000CF3FD10519F010F0CFEFD0E080912039B4
:1047400070E060E08111BE018AEA91E00E943305C9
:104750000EE215E3C8018E5295438C179D07B0F603
:10476000F80161918F018AEA91E00E94B100F2CFD5
:1047700082E00E947B1E85E090E0DF91CF911F9147
:104780000F91FF90EF90DF90CF900C9448180F930B
:104790001F93CF93DF938091C90181116EC081E097
:1047A0008093C901C0E0D8E14FB7F8942091021D71
:1047B0003091031D8091041D9091051D4FBF281756
:1047C000390709F45AC0E091021DF091031D809150
:1047D000001D9091011DE817F90709F03FC0809175
:1047E000FE1C9091FF1C9093031D8093021D00817D
:1047F0001181E091681BF091691B2091661B30913B
:10480000671BE217F30789F52091641B3091651B44
:104810003093691B2093681B20813181A90141508D
:104820005109443F514008F0BFCFEEE2F5E30E528C
:104830001543C8018E0F9F1FBE010E94192EDC0177
:10484000AE52BE4F8C918193CF018E529543821709
:10485000930778F3C9010E943123A6CFE091021D8E
:10486000F091031DCF010296BECFE091681BF0913D
:10487000691B9F012E5F3F4FCBCF1092D101109249
:10488000D0011092CF011092C901DF91CF911F91F9
:104890000F910895809123398823E1F10E944E1DE4
:1048A0008091D101882311F180912035811102C0BE
:1048B0000E94F21C80912235811128C080912135FF
:1048C000811124C080912035882331F062E370E0AB
:1048D00080E090E00E94D7280E94F21C809122354F
:1048E000811104C0109220350E94C7234FB7F8945D
:1048F00020910B3530910C3580910D3590910E350E
:104900004FBF2817390791F00C94122281E0809351
:104910002035ECCF80912239882319F00E94E718C6
:10492000E5CF0E942A190E94AF1CE0CF0895CF93D3
:104930008091CA01811127C081E08093CA01C4E13E
:104940008BE399E30E94902A892BD9F08FB7F894D2
:1049500040910B3550910C35209107353091083539
:104960004217530791F440910D3550910E35209127
:10497000093530910A354217530739F48FBFC150BA
:10498000F9F61092CA01CF91089540910D355091DA
:104990000E3520910B3530910C35215031094217DD
:1049A000530761F38FBF8BE399E30E94AA2A2FB7C5
:1049B000F894E0910D35F0910E35808340910D35DE
:1049C00050910E358091093590910A354817590755
:1049D00051F4809107359091083590930E3580936E
:1049E0000D352FBFCCCF80910D3590910E350196AE
:1049F000F4CF1F920F920FB60F9211240BB60F92A5
:104A00002F933F934F935F936F937F938F939F93D6
:104A1000AF93BF93EF93FF930E949724FF91EF9181
:104A2000BF91AF919F918F917F916F915F914F91C6
:104A30003F912F910F900BBE0F900FBE0F901F90C4
:104A400018958091DC3980FF2AC082E0809315356B
:104A50008091153581508230B8F50E94031B882360
:104A600081F10E941A1B882361F10E94271B882371
:104A700041F10E94361B882321F10E94431B8823A9
:104A800051F181E0809322390E94891B882319F11A
:104A90000E94931B82E1809314010C94AD1E82FF4F
:104AA00002C083E0D3CF83FF02C081E0CFCF42E2D8
:104AB00050E065E571E08BE399E30E945A2C0E9477
:104AC0007E18109222390895109222394EE150E05A
:104AD00068E771E0F0CF089580E00E9458290E94B5
:104AE0008D2CA6E0BDE181E098E1FD019C011192D1
:104AF00021503040E1F7E7E0F5E3B183A083B783CD
:104B0000A683B583A48386E095E39383828326E01E
:104B100040E052EC61E070E08BE399E30E94612B8E
:104B20000E94721D61E08CE00E94262A61E08DE007
:104B30000E94262AE6E2F7E384EF91E0DF019C0180
:104B40001D9221503040E1F7E2E2F7E384E0DF011B
:104B50001D928A95E9F7E2EDF1E080E098E1DF014E
:104B60009C011D9221503040E1F7ACE6BBE182E9A7
:104B700091E0FD019C01119221503040E1F7EEEFF0
:104B8000FCE1B183A083B783A683B583A4832CEF14
:104B90003CE133832283A2EDB9E1FD019C01119236
:104BA00021503040E1F7E4E6FBE1B183A083B78315
:104BB000A683B583A48382E69BE19383828322E06C
:104BC00030E043E050E064E070E08AEA91E00E9467
:104BD000F7000C942125CF93CFB7F8948091313909
:104BE000811127C0E0EDF0E08491E0EBF0E09491DA
:104BF000E82FF0E0EE0FFF1FEA50FF4FA591B491B0
:104C0000EC91E92321F461E084E00E94622A61E0F2
:104C100084E00E94262A8CB580618CBD8CB58064AE
:104C20008CBD61E087E00E94262A61E085E00E9459
:104C3000262A809131398F5F80933139CFBFCF9150
:104C400008959FB7F89480913139882319F08150E5
:104C50008093313980913139811105C08CB58F7BBA
:104C60008CBD109230399FBF08952FB7F8948130D2
:104C700041F0C0F08230A1F082E08093303980E0D2
:104C800001C082E090912F39892B80932F39809138
:104C90003039811103C081E0809330392FBF0895EE
:104CA00084E0F0CF81E0EECF909130399230A1F0E6
:104CB0009FB7F894833088F4E82FF0E0E956FE4F70
:104CC0008081809520912F39822380932F39811103
:104CD00002C0109230399FBF089580E0F2CF08954E
:104CE000833060F5E82FF0E0EE0FFF1FE65EFE4F29
:104CF00071836083813051F08230A1F0809169002E
:104D00008C7F482B40936900E89A08958091690050
:104D1000837F440F551F440F551F482B4093690054
:104D2000E99A0895809169008F7C94E0440F551FA3
:104D30009A95E1F7482B40936900EA9A08958330E9
:104D400078F4E82FF0E0813061F0823061F0E8988B
:104D5000EE0FFF1FE65EFE4F8FE696E291838083A3
:104D60000895E998F5CFEA98F3CF1F920F920FB606
:104D70000F9211240BB60F922F933F934F935F9393
:104D80006F937F938F939F93AF93BF93EF93FF9313
:104D9000E0911A01F0911B010995FF91EF91BF91EC
:104DA000AF919F918F917F916F915F914F913F91C3
:104DB0002F910F900BBE0F900FBE0F901F90189564
:104DC0001F920F920FB60F9211240BB60F922F93D2
:104DD0003F934F935F936F937F938F939F93AF9383
:104DE000BF93EF93FF93E0911C01F0911D01099592
:104DF000FF91EF91BF91AF919F918F917F916F91B3
:104E00005F914F913F912F910F900BBE0F900FBE6E
:104E10000F901F9018951F920F920FB60F921124AA
:104E20000BB60F922F933F934F935F936F937F93A4
:104E30008F939F93AF93BF93EF93FF93E0911E01E6
:104E4000F0911F010995FF91EF91BF91AF919F9153
:104E50008F917F916F915F914F913F912F910F9023
:104E60000BBE0F900FBE0F901F9018950F931F93BE
:104E7000CF93DF938230910510F482E090E0E091CF
:104E8000DA39F091DB3930E020E0B0E0A0E0309793
:104E900099F42115310509F44AC0281B390B243037
:104EA0003105D8F58A819B816115710589F1FB0176
:104EB00093838283FE0111C040815181028113815D
:104EC00048175907E0F04817590799F4109761F00F
:104ED00012960C93129713961C933296CF01DF9182
:104EE000CF911F910F9108950093DA391093DB3918
:104EF000F4CF2115310551F04217530738F0A901BD
:104F0000DB019A01BD01DF01F801C1CFEF01F9CF4B
:104F10009093DB398093DA39CDCFFE01E20FF31F96
:104F2000819391932250310939832883D7CF2091DF
:104F3000D8393091D939232B41F420912201309175
:104F400023013093D9392093D83920912001309111
:104F500021012115310541F42DB73EB740912401BF
:104F600050912501241B350BE091D839F091D939A6
:104F7000E217F307A0F42E1B3F0B2817390778F030
:104F8000AC014E5F5F4F2417350748F04E0F5F1F8F
:104F90005093D9394093D839819391939FCFF0E0C2
:104FA000E0E09CCFCF93DF930097E9F0FC013297CC
:104FB00013821282A091DA39B091DB39ED0130E031
:104FC00020E01097A1F420813181820F931F20915E
:104FD000D8393091D9392817390709F061C0F093D1
:104FE000D939E093D839DF91CF910895EA01CE17EE
:104FF000DF07E8F54A815B819E0141155105B1F754
:10500000E901FB83EA8349915991C40FD51FEC173D
:10501000FD0761F4808191810296840F951FE9015B
:1050200099838883828193819B838A83F0E0E0E087
:1050300012968D919C9113970097B9F52D913C9103
:105040001197CD010296820F931F2091D83930918C
:10505000D9392817390739F6309751F51092DB39CD
:105060001092DA39B093D939A093D839BCCFD38311
:10507000C28340815181840F951FC817D90761F4FD
:105080004E5F5F4F88819981480F591F518340833C
:105090008A819B81938382832115310509F0B0CFEA
:1050A000F093DB39E093DA399ECFFD01DC01C0CF0C
:1050B00013821282D7CF08951F920F920FB60F92CC
:1050C00011242F933F938F939F93AF93BF9380911E
:1050D000333990913439A0913539B09136393091C6
:1050E000323923E0230F2D3758F50196A11DB11D4C
:1050F000209332398093333990933439A0933539E2
:10510000B09336398091373990913839A091393937
:10511000B0913A390196A11DB11D80933739909312
:105120003839A0933939B0933A39BF91AF919F91F3
:105130008F913F912F910F900FBE0F901F90189558
:1051400026E8230F0296A11DB11DD2CF2FB7F894E8
:105150006091333970913439809135399091363975
:105160002FBF08953FB7F89480913739909138391F
:10517000A0913939B0913A3926B5A89B05C02F3F87
:1051800019F00196A11DB11D3FBFBA2FA92F982F6D
:105190008827BC01CD01620F711D811D911D42E068
:1051A000660F771F881F991F4A95D1F708958F9230
:1051B0009F92AF92BF92CF92DF92EF92FF926B01DC
:1051C0007C010E94B2284B015C01C114D104E104AE
:1051D000F104E9F00E945B280E94B228681979095D
:1051E0008A099B09683E73408105910570F321E0AF
:1051F000C21AD108E108F10888EE880E83E0981EF3
:10520000A11CB11CC114D104E104F10429F7FF90E1
:10521000EF90DF90CF90BF90AF909F908F900895C8
:10522000789484B5826084BD84B5816084BD85B581
:10523000826085BD85B5816085BDEEE6F0E0808148
:1052400081608083E1E8F0E0108280818260808369
:10525000808181608083E0E8F0E0808181608083EC
:10526000E1EBF0E0808184608083E0EBF0E080811E
:1052700081608083E1E9F0E08081826080838081C9
:1052800081608083E0E9F0E0808181608083EAE7EB
:10529000F0E080818460808380818260808380816F
:1052A000816080838081806880831092C10008952E
:1052B000883020F0873108F487E188512091260159
:1052C00090E4299F900111248770822B80937C00A9
:1052D00080917A00806480937A0080917A0086FDC4
:1052E000FCCF809178009091790008951F93CF931F
:1052F000DF93182FEB0161E00E94262A209739F4F2
:1053000060E0812FDF91CF911F910C94622ACF3FF3
:10531000D10511F461E0F5CFE12FF0E0E457FF4F44
:10532000E491E150EA3008F054C0F0E0E656F64D62
:105330000C946E2EA429AC29B129BB29E929E929AD
:10534000C529CD29D529DF2984B5806884BDC7BD8D
:10535000DF91CF911F91089584B5806284BDC8BD4F
:10536000F7CF80918000806880938000D09389007F
:10537000C0938800EDCF8091800080628093800090
:10538000D0938B00C0938A00E3CF8091B0008068F7
:105390008093B000C093B300DBCF8091B0008062F7
:1053A0008093B000C093B400D3CF80919000806808
:1053B00080939000D0939900C0939800C9CF8091BA
:1053C0009000806280939000D0939B00C0939A00DD
:1053D000BFCFC038D1050CF09DCF92CF81508A301D
:1053E00080F5E82FF0E0E950F64D0C946E2E0B2A74
:1053F0000F2A012A072A212A212A122A182A1C2ABE
:10540000222A809180008F77809380000895809178
:1054100080008F7DF9CF84B58F7784BD089584B5E2
:105420008F7DFBCF8091B0008F778093B00008957F
:105430008091B0008F7DF9CF809190008F7780931D
:1054400090000895809190008F7DF9CFCF93DF93E6
:1054500090E0FC01E455FF4F249184539F4FFC01E1
:1054600084918823C9F090E0880F991FFC01EA50CD
:10547000FF4FA591B491FC01E451FF4FC591D49128
:1054800061110DC09FB7F8948C91209582238C9365
:105490008881282328839FBFDF91CF9108956230B0
:1054A00051F49FB7F8943C91822F809583238C937D
:1054B000E8812E2BEFCF8FB7F894EC912E2B2C9305
:1054C0008FBFEACF1F93CF93DF93282F30E0F901EE
:1054D000E457FF4F8491F901E455FF4FD491F9014E
:1054E000E453FF4FC491CC23A9F0162F81110E94E1
:1054F000EE29EC2FF0E0EE0FFF1FE451FF4FA591D6
:10550000B4918FB7F894EC91111108C0D095DE23B7
:10551000DC938FBFDF91CF911F910895DE2BF8CFE1
:10552000FC01918D228D892F90E0805C9F4F821B22
:1055300091098F7399270895FC01918D828D981799
:1055400031F0828DE80FF11D858D90E008958FEF89
:105550009FEF0895FC01918D828D981761F0A28DC7
:10556000AE0FBF2FB11D5D968C91928D9F5F9F7383
:10557000928F90E008958FEF9FEF089583E29CE271
:10558000892B49F080E090E0892B29F00E94232CA0
:1055900081110E94000080E090E0892B49F080E0BA
:1055A00090E0892B29F00E94000081110C940000EA
:1055B0000895FC01A48DA80FB92FB11DA35ABF4FA8
:1055C0002C91848D90E001968F739927848FA68902
:1055D000B7892C93A089B1898C9180648C93938D29
:1055E000848D981306C00288F389E02D80818F7D19
:1055F00080830895CF93DF93EC01888D8823B9F0E1
:10560000AA89BB89E889F9898C9185FD03C08081CD
:1056100086FD0DC00FB607FCF7CF8C9185FFF2CF4A
:10562000808185FFEDCFCE010E94D92AE9CFDF919D
:10563000CF910895EF92FF920F931F93CF93DF9333
:10564000EC0181E0888F9B8D8C8D981316C0E889C2
:10565000F989808185FF11C0EE89FF896083E8891F
:10566000F98980818064808381E090E0DF91CF912F
:105670001F910F91FF90EF900895F62E0B8D10E083
:105680000F5F1F4F0F731127E02E8C8D8E110CC0F2
:105690000FB607FCFACFE889F989808185FFF5CF3D
:1056A000CE010E94D92AF1CFEB8DEC0FFD2FF11D19
:1056B000E35AFF4FF0820B8FEA89FB898081806279
:1056C000D2CFCF92DF92EF92FF921F93CF93DF93CF
:1056D000EC016A017B01122FE889F98982E080835D
:1056E000C11481EED806E104F104A1F060E079E094
:1056F0008DE390E0A70196010E942D2E21503109E3
:10570000410951095695479537952795211580E10F
:10571000380798F0E889F989108260E874E88EE12A
:1057200090E0A70196010E942D2E215031094109D8
:1057300051095695479537952795EC85FD8530831A
:10574000EE85FF852083188EEC89FD891083EA8918
:10575000FB89808180618083EA89FB898081886000
:105760008083EA89FB89808180688083EA89FB895C
:1057700080818F7D8083DF91CF911F91FF90EF908B
:10578000DF90CF9008951F920F920FB60F921124C1
:105790000BB60F922F938F939F93EF93FF93E0910C
:1057A0004B39F0914C398081E0915139F091523967
:1057B00082FD1DC09081809154398F5F8F7320913D
:1057C0005539821741F0E0915439F0E0E55CF64C30
:1057D000958F80935439FF91EF919F918F912F91E5
:1057E0000F900BBE0F900FBE0F901F9018958081E9
:1057F000F2CF1F920F920FB60F9211240BB60F9299
:105800002F933F934F935F936F937F938F939F93C8
:10581000AF93BF93EF93FF938BE399E30E94D92A51
:10582000FF91EF91BF91AF919F918F917F916F9178
:105830005F914F913F912F910F900BBE0F900FBE34
:105840000F901F9018958BE399E30E94902A21E016
:10585000892B09F420E0822F0895EBE3F9E313820A
:10586000128288EE93E0A0E0B0E084839583A68363
:10587000B7838EE991E09183808385EC90E09587F2
:10588000848784EC90E09787868780EC90E0918B0A
:10589000808B81EC90E0938B828B82EC90E0958BF7
:1058A000848B86EC90E0978B868B118E128E138EF4
:1058B000148E0895AF92BF92CF92DF92EF92FF9233
:1058C0000F931F93CF93DF936C017B018B01040F28
:1058D000151FEB015E01AE18BF08C017D10759F0C4
:1058E0006991D601ED91FC910190F081E02DC60106
:1058F0000995892B79F7C501DF91CF911F910F9100
:10590000FF90EF90DF90CF90BF90AF900895FC0193
:1059100044835583668377830895009729F0BC01FB
:1059200090E080E00C94FC2F0895CF92DF92EF92EC
:10593000FF926B017C01C114D104E104F10441F038
:105940000E94AD2FA70196010E944F2E6B017C0192
:10595000C701B601FF90EF90DF90CF9008950895B2
:105960000E9410290E94AF2C0E946C25CEEBDAE237
:105970000E944A242097E1F30E94BE2AF9CF0E9498
:10598000372D08F481E008950E94CB2C6894B11162
:105990000C94A62D08950E948B2D88F09F5798F0A7
:1059A000B92F9927B751B0F0E1F0660F771F881F24
:1059B000991F1AF0BA95C9F714C0B13091F00E943E
:1059C000A52DB1E008950C94A52D672F782F882779
:1059D000B85F39F0B93FCCF3869577956795B39565
:1059E000D9F73EF490958095709561957F4F8F4FD4
:1059F0009F4F0895E89409C097FB3EF490958095D9
:105A0000709561957F4F8F4F9F4F9923A9F0F92F84
:105A100096E9BB279395F695879577956795B79502
:105A2000F111F8CFFAF4BB0F11F460FF1BC06F5FE8
:105A30007F4F8F4F9F4F16C0882311F096E911C0FA
:105A4000772321F09EE8872F762F05C0662371F01B
:105A500096E8862F70E060E02AF09A95660F771F2F
:105A6000881FDAF7880F9695879597F90895990F0B
:105A70000008550FAA0BE0E8FEEF16161706E80718
:105A8000F907C0F012161306E407F50798F0621B39
:105A9000730B840B950B39F40A2661F0232B242B0E
:105AA000252B21F408950A2609F4A140A6958FEF2D
:105AB000811D811D089597F99F6780E870E060E07F
:105AC00008959FEF80EC089500240A941616170697
:105AD00018060906089500240A94121613061406DF
:105AE00005060895092E0394000C11F4882352F042
:105AF000BB0F40F4BF2B11F460FF04C06F5F7F4FFA
:105B00008F4F9F4F089557FD9058440F551F59F0E0
:105B10005F3F71F04795880F97FB991F61F09F3F9A
:105B200079F087950895121613061406551FF2CFC3
:105B30004695F1DF08C0161617061806991FF1CF13
:105B400086957105610508940895E894BB2766273A
:105B50007727CB0197F908950E94BF2D0C94722DE1
:105B60000E94642D38F00E946B2D20F0952311F0D7
:105B70000C945B2D0C94612D11240C94A62D0E9485
:105B8000832D70F3959FC1F3950F50E0551F629FD1
:105B9000F001729FBB27F00DB11D639FAA27F00D86
:105BA000B11DAA1F649F6627B00DA11D661F829FAD
:105BB0002227B00DA11D621F739FB00DA11D621F92
:105BC000839FA00D611D221F749F3327A00D611DAF
:105BD000231F849F600D211D822F762F6A2F112491
:105BE0009F5750409AF0F1F088234AF0EE0FFF1FC4
:105BF000BB1F661F771F881F91505040A9F79E3F1B
:105C0000510580F00C945B2D0C94A62D5F3FE4F3BE
:105C1000983ED4F3869577956795B795F795E79570
:105C20009F5FC1F7FE2B880F911D9695879597F979
:105C30000895AA1BBB1B51E107C0AA1FBB1FA617D3
:105C4000B70710F0A61BB70B881F991F5A95A9F725
:105C500080959095BC01CD010895A1E21A2EAA1B52
:105C6000BB1BFD010DC0AA1FBB1FEE1FFF1FA2170C
:105C7000B307E407F50720F0A21BB30BE40BF50B09
:105C8000661F771F881F991F1A9469F76095709592
:105C9000809590959B01AC01BD01CF010895052E23
:105CA00097FB1EF400940E94662E57FD07D00E94B9
:105CB0002D2E07FC03D04EF40C94662E5095409583
:105CC000309521953F4F4F4F5F4F089590958095A8
:105CD000709561957F4F8F4F9F4F0895EE0FFF1F77
:105CE0000024001C0BBE0790F691E02D0994692753
:105CF0009627692778278727782708950E94492FB4
:105D0000A59F900DB49F900DA49F800D911D11240F
:105D10000895E894DF93CF93FC01DB010E94492FA3
:105D20007F936F93E9019A01AC01BF93AF933F93C7
:105D30002F93DF010E94492F26F46C1B7D0B820BF1
:105D4000930B9E01EB01FC010E94582FAF91BF9174
:105D50002F913F910E94582FBE01CF01F9012F9141
:105D60003F91CF91DF910895689401C0E8948F929C
:105D70009F92CF93DF930E94C22EDF91CF919F908D
:105D80008F90089588249924F401E401B0E49F934E
:105D9000AA279A158B049C04ED05FE05CF05D007B4
:105DA000A10798F4AD2FDC2FCF2FFE2FE92D982CD3
:105DB000892E982F872F762F652F542F432F322F20
:105DC0002227B85031F7BF9127C01B2EBF91BB27A8
:105DD000220F331F441F551F661F771F881F991FEF
:105DE000881C991CEE1FFF1FCC1FDD1FAA1FBB1FA5
:105DF0008A149B04EC05FD05CE05DF05A007B1075D
:105E000048F08A189B08EC09FD09CE09DF09A00BB0
:105E1000B10B21601A94E1F62EF49401AF01BE019A
:105E2000CD01000C0895002E083090F0982F872F98
:105E3000762F652F542F432F322F22270850F4CF6F
:105E4000220F331F441F551F661F771F881F991F7E
:105E50000A95B2F7002D089597FD1094002E083092
:105E600098F00850232F342F452F562F672F782F67
:105E7000892F912DF4CF15949795879577956795F0
:105E800057954795379527950A95AAF71124002D20
:105E90000895A29FB001B39FC001A39F700D811D03
:105EA0001124911DB29F700D811D1124911D089523
:105EB0000E94492F460F571FC81FD91F08F431965B
:105EC00008958F929F92AF92BF92CF92DF92EF92FE
:105ED000FF92CF93DF93EC01688179818A819B8166
:105EE000611571058105910521F464E279ED8BE579
:105EF00097E02DE133EF41E050E00E944F2E490141
:105F00005A019B01AC01A7EAB1E40E947E2E6B010D
:105F10007C01ACEEB4EFA50194010E942E30C60EB8
:105F2000D71EE81EF91EF7FE06C081E0C81AD10888
:105F3000E10880E8F80AC882D982EA82FB82C701B8
:105F4000B6019F77DF91CF91FF90EF90DF90CF90D8
:105F5000BF90AF909F908F9008958F929F92AF9235
:105F6000BF92CF92DF92EF92FF9260910001709109
:105F70000101809102019091030161157105810574
:105F8000910521F464E279ED8BE597E02DE133EFA3
:105F900041E050E00E944F2E49015A019B01AC01A3
:105FA000A7EAB1E40E947E2E6B017C01ACEEB4EF57
:105FB000A50194010E942E30C60ED71EE81EF91EC0
:105FC000F7FE06C081E0C81AD108E10880E8F80AA7
:105FD000C0920001D0920101E0920201F09203010F
:105FE000C701B6019F77FF90EF90DF90CF90BF90F1
:105FF000AF909F908F90089560930001709301017E
:1060000080930201909303010895FB01DC0102C01B
:1060100001900D9241505040D8F70895DC0101C025
:106020006D9341505040E0F70895F999FECF92BD2D
:1060300081BDF89A992780B50895262FF999FECF4A
:106040001FBA92BD81BD20BD0FB6F894FA9AF99A95
:106050000FBE01960895B7FF0C947E2E0E947E2EEF
:0A606000821B930B0895F894FFCF04
:10606A0001000000F82A00002801FE030000000FCA
:10607A0000FFDCFE1101FF0005006F266F266F2668
:10608A000000DD39800001781E00A02800F03C00E5
:10609A00405100127A00E4A20024F40048E801907A
:1060AA00D00320A10700000000B1004502B101BFE2
:1060BA00018002C7004572726F722C20696E646596
:1060CA007465726D696E61746520626F6F74207693
:1060DA006563746F720D0A004572726F722C2069C3
:1060EA006E636F727265637420626F6F7420766577
:1060FA0063746F720D0A00010204000000001A2B7B
:0A610A005A2C902AAA2A9C2AFA2A8D
:00000001FF
